:100000008A110A120528000009000730990083169A
:100010000510851005118515831205108510E8302F
:10002000A0000330A1004E20851D1B28C830A00071
:10003000A1014E2014281F30830505148519252899
:10004000C830A000A1014E201E281F3083050530B6
:1000500084000230AA009930A0000230A10096303E
:10006000A2000030A30089205030A000A1014E2042
:10007000053084000230AA009930A0000230A100AF
:100080004B30A2000030A30089202C30A0000130AA
:10009000A1004E20051014284C284D28A008031953
:1000A00059286020A00300000000000000000000AC
:1000B0004E28A108031908006020A103A0034E28C0
:1000C0000C30A500A50B6228000000001230A20031
:1000D000A20B6F2871207120000000000800712021
:1000E00068280D30A400A40B73280000080010300D
:1000F000A8020001031C013EA902031C080080287D
:100100000A30A8020001031C013EA902031C0800DA
:1001100080282A0880042008A8002108A900772048
:100120000130A202031CA3032A0980052008A800AD
:100130002108A9007720A208031D8928A308031D10
:040140008928080002
:02400E00C431BB
:00000001FF
